:100000000C9434000C9451000C9451000C94510049
:100010000C9451000C9451000C9451000C9451001C
:100020000C9451000C9451000C9451000C9451000C
:100030000C9451000C9451000C9451000C945100FC
:100040000C9451000C9451000C9451000C945100EC
:100050000C9451000C9451000C9451000C945100DC
:100060000C9451000C94510011241FBECFEFD8E026
:10007000DEBFCDBF11E0A0E0B1E0E2E6FBE002C0F0
:1000800005900D92A433B107D9F721E0A4E3B1E0C4
:1000900001C01D92A839B207E1F70E94BE000C947E
:1000A000AF050C940000389839983A983B983C98E2
:1000B0003D9852985398549A559A569A579A219A1D
:1000C000229A299A5F9A2A98519A5098089520E086
:1000D00030E040E851E40E947B029B01AC0160E00B
:1000E00074E284E79BE40E94910120E030E040E864
:1000F0005FE30E942C010E94F9017093C500609398
:10010000C40088E98093C10086E08093C20008950E
:10011000E0ECF0E0908195FFFDCF8093C60008955C
:10012000CF93DF93EC018881882331F021960E94E0
:10013000880089918111FBCFDF91CF91089596B10D
:1001400066B146B186B156B156B159B159B1627076
:1001500070E0660F771F292F217030E0262B372B98
:10016000447050E0440F551F440F551F242B352B6E
:100170008870880F880F880F822B08950E94530083
:100180002FEF89E698E1215080409040E1F700C0D0
:10019000000060E070E086E196E40E9467002FEFC7
:1001A00089E698E1215080409040E1F700C00000CE
:1001B00080E091E00E9490002FEF87EA91E62150C5
:1001C00080409040E1F700C000000CE111E0C4E382
:1001D000D1E05C985D985E9A8FE39CE90197F1F716
:1001E00000C000000E949F005D9A8FE39CE9019788
:1001F000F1F700C000000E949F005D985E988FE3B9
:100200009CE90197F1F700C000000E949F005D9AF1
:100210008FE39CE90197F1F700C000000E949F0066
:100220005C9A1F928F931F930F93DF93CF930E943B
:10023000DE02CE010E9490008FEF91EE24E081500B
:1002400090402040E1F700C000000F900F900F9009
:100250000F900F900F90BDCF5058BB27AA270ED0FC
:1002600010C101D130F006D120F031F49F3F11F4DC
:100270001EF4F6C00EF4E095E7FBECC0E92F12D1B6
:1002800080F3BA17620773078407950718F071F4B3
:100290009EF52AC10EF4E0950B2EBA2FA02D0B016E
:1002A000B90190010C01CA01A0011124FF27591BBB
:1002B00099F0593F50F4503E68F11A16F040A22FC1
:1002C000232F342F4427585FF3CF46953795279532
:1002D000A795F0405395C9F77EF41F16BA0B620B31
:1002E000730B840BBAF09150A1F0FF0FBB1F661F78
:1002F000771F881FC2F70EC0BA0F621F731F841FBB
:1003000048F4879577956795B795F7959E3F08F0E0
:10031000B3CF9395880F08F09927EE0F979587959F
:1003200008950CD0AEC0A6D040F09DD030F021F49E
:100330005F3F19F08FC05111D8C092C0B3D098F36D
:100340009923C9F35523B1F3951B550BBB27AA2756
:1003500062177307840738F09F5F5F4F220F331FC8
:10036000441FAA1FA9F333D00E2E3AF0E0E830D094
:1003700091505040E695001CCAF729D0FE2F27D097
:10038000660F771F881FBB1F261737074807AB0765
:10039000B0E809F0BB0B802DBF01FF2793585F4FDA
:1003A0002AF09E3F510568F055C09FC05F3FECF3B7
:1003B000983EDCF3869577956795B795F7959F5F9F
:1003C000C9F7880F911D9695879597F90895E1E0F3
:1003D000660F771F881FBB1F621773078407BA0752
:1003E00020F0621B730B840BBA0BEE1F88F7E095AD
:1003F000089504D06894B11178C008955BD088F056
:100400009F5790F0B92F9927B751A0F0D1F0660F00
:10041000771F881F991F1AF0BA95C9F712C0B1301B
:1004200081F062D0B1E008955FC0672F782F8827F0
:10043000B85F39F0B93FCCF3869577956795B3955A
:10044000D9F73EF490958095709561957F4F8F4FC9
:100450009F4F089597F99F6780E870E060E00895E6
:100460009FEF80EC089500240A94161617061806CC
:100470000906089500240A941216130614060506A8
:100480000895092E0394000C11F4882352F0BB0F39
:1004900040F4BF2B11F460FF04C06F5F7F4F8F4F9C
:1004A0009F4F089557FD9058440F551F59F05F3FD7
:1004B00071F04795880F97FB991F61F09F3F79F086
:1004C00087950895121613061406551FF2CF469508
:1004D000F1DF08C0161617061806991FF1CF86958A
:1004E0007105610508940895E894BB27662777276E
:1004F000CB0197F908950BD0C4CFB5DF28F0BADF50
:1005000018F0952309F0A6CFABCF1124EECFCADFA8
:10051000A0F3959FD1F3950F50E0551F629FF00116
:10052000729FBB27F00DB11D639FAA27F00DB11D6F
:10053000AA1F649F6627B00DA11D661F829F2227F8
:10054000B00DA11D621F739FB00DA11D621F839F7F
:10055000A00D611D221F749F3327A00D611D231F55
:10056000849F600D211D822F762F6A2F11249F57A3
:1005700050408AF0E1F088234AF0EE0FFF1FBB1FC6
:10058000661F771F881F91505040A9F79E3F510565
:1005900070F060CFAACF5F3FECF3983EDCF3869516
:1005A00077956795B795F795E7959F5FC1F7FE2B10
:1005B000880F911D9695879597F90895AEE0B0E064
:1005C000E4EEF2E00C9486050D891E8986E08C83AA
:1005D0001A8309838FEF9FE79E838D83AE01475E69
:1005E0005F4F6F89788DCE0101960E940003EF81E5
:1005F000F885E00FF11F10822E96E4E00C94A2051E
:10060000ACE0B0E0E6E0F3E00C9478057C016B012F
:100610008A01FC0117821682838181FFBDC1CE0150
:1006200001964C01F7019381F60193FD859193FFAB
:1006300081916F01882309F4ABC1853239F493FDB0
:10064000859193FF81916F01853229F4B70190E084
:100650000E94E804E7CF512C312C20E02032A0F496
:100660008B3269F030F4803259F0833269F42061C2
:100670002CC08D3239F0803339F4216026C02260DD
:10068000246023C0286021C027FD27C030ED380F2B
:100690003A3078F426FF06C0FAE05F9E300D112450
:1006A000532E13C08AE0389E300D1124332E206261
:1006B0000CC08E3221F426FD6BC1206406C08C363E
:1006C00011F4206802C0883641F4F60193FD85914B
:1006D00093FF81916F018111C1CF982F9F7D955418
:1006E000933028F40C5F1F4FFFE3F9830DC083366E
:1006F00031F0833771F0833509F05BC022C0F80117
:10070000808189830E5F1F4F44244394512C5401F0
:1007100015C03801F2E06F0E711CF801A080B180A5
:1007200026FF03C0652D70E002C06FEF7FEFC501AB
:100730002C870E94DD042C0183012C852F77222E2B
:1007400017C03801F2E06F0E711CF801A080B18073
:1007500026FF03C0652D70E002C06FEF7FEFC5017B
:100760002C870E94D2042C012C852068222E830124
:1007700023FC1BC0832D90E048165906B0F4B70146
:1007800080E290E00E94E8043A94F4CFF50127FC5F
:10079000859127FE81915F01B70190E00E94E804F6
:1007A00031103A94F1E04F1A51084114510471F795
:1007B000E5C0843611F0893639F5F80127FF07C006
:1007C00060817181828193810C5F1F4F08C06081BD
:1007D0007181882777FD8095982F0E5F1F4F2F76A8
:1007E000B22E97FF09C090958095709561957F4FC7
:1007F0008F4F9F4F2068B22E2AE030E0A4010E9464
:100800001A05A82EA81844C0853729F42F7EB22EC9
:100810002AE030E025C0F22FF97FBF2E8F36C1F0DD
:1008200018F4883579F0B4C0803719F0883721F092
:10083000AFC02F2F2061B22EB4FE0DC08B2D84606F
:10084000B82E09C024FF0AC09F2F9660B92E06C09B
:1008500028E030E005C020E130E002C020E132E0D5
:10086000F801B7FE07C060817181828193810C5FBE
:100870001F4F06C06081718180E090E00E5F1F4FC6
:10088000A4010E941A05A82EA818FB2DFF77BF2EE1
:10089000B6FE0BC02B2D2E7FA51450F4B4FE0AC05B
:1008A000B2FC08C02B2D2E7E05C07A2C2B2D03C048
:1008B0007A2C01C0752C24FF0DC0FE01EA0DF11D3C
:1008C0008081803311F4297E09C022FF06C0739411
:1008D000739404C0822F867809F0739423FD13C0AB
:1008E00020FF06C05A2C731418F4530C5718732C9D
:1008F000731468F4B70180E290E02C870E94E8044A
:1009000073942C85F5CF731410F4371801C0312C73
:1009100024FF12C0B70180E390E02C870E94E80416
:100920002C8522FF17C021FF03C088E590E002C09C
:1009300088E790E0B7010CC0822F867859F021FD3E
:1009400002C080E201C08BE227FD8DE2B70190E09A
:100950000E94E804A51438F4B70180E390E00E94F7
:10096000E8045A94F7CFAA94F401EA0DF11D8081AE
:10097000B70190E00E94E804A110F5CF332009F4FC
:1009800051CEB70180E290E00E94E8043A94F6CF9D
:10099000F7018681978102C08FEF9FEF2C96E2E1ED
:1009A0000C949405FC010590615070400110D8F73B
:1009B000809590958E0F9F1F0895FC0161507040A7
:1009C00001900110D8F7809590958E0F9F1F089584
:1009D0000F931F93CF93DF93182F092FEB018B8178
:1009E00081FD03C08FEF9FEF20C082FF10C04E81BA
:1009F0005F812C813D81421753077CF4E881F981A6
:100A00009F012F5F3F4F39832883108306C0E885FD
:100A1000F985812F0995892B29F72E813F812F5F39
:100A20003F4F3F832E83812F902FDF91CF911F91D6
:100A30000F910895FA01AA27283051F1203181F150
:100A4000E8946F936E7F6E5F7F4F8F4F9F4FAF4FD6
:100A5000B1E03ED0B4E03CD0670F781F891F9A1FE9
:100A6000A11D680F791F8A1F911DA11D6A0F711D9D
:100A7000811D911DA11D20D009F468943F912AE0A9
:100A8000269F11243019305D3193DEF6CF01089591
:100A9000462F4770405D4193B3E00FD0C9F7F6CFC2
:100AA000462F4F70405D4A3318F0495D31FD40528A
:100AB000419302D0A9F7EACFB4E0A6959795879520
:100AC00077956795BA95C9F70097610571050895FF
:100AD0009B01AC010A2E06945795479537952795AB
:100AE000BA95C9F7620F731F841F951FA01D089543
:100AF0002F923F924F925F926F927F928F929F922E
:100B0000AF92BF92CF92DF92EF92FF920F931F931B
:100B1000CF93DF93CDB7DEB7CA1BDB0B0FB6F894CC
:100B2000DEBF0FBECDBF09942A88398848885F840C
:100B30006E847D848C849B84AA84B984C884DF807D
:100B4000EE80FD800C811B81AA81B981CE0FD11D61
:100B50000FB6F894DEBF0FBECDBFED010895F89437
:020B6000FFCFC5
:100B620044657669636520496E697469616C697A66
:100B720065642121210D0A0D0A0D0A0054686520C1
:100B82006C73622076616C75652069733A20256406
:040B92002E0D0A001A
:00000001FF
